 redefclass004

 Timestamp is 86806870 (reproducible build file hash)

 Preferred load address is 0000000180000000

 Start         Length     Name                   Class
 0001:00000000 00002d80H .text$mn                CODE
 0001:00002d80 00000036H .text$mn$00             CODE
 0001:00002db6 00000092H .text$x                 CODE
 0002:00000000 00000198H .idata$5                DATA
 0002:00000198 00000038H .00cfg                  DATA
 0002:000001d0 00000008H .CRT$XCA                DATA
 0002:000001d8 00000008H .CRT$XCZ                DATA
 0002:000001e0 00000008H .CRT$XIA                DATA
 0002:000001e8 00000008H .CRT$XIC                DATA
 0002:000001f0 00000008H .CRT$XIZ                DATA
 0002:000001f8 00000008H .CRT$XLA                DATA
 0002:00000200 00000008H .CRT$XLZ                DATA
 0002:00000208 00000008H .CRT$XPA                DATA
 0002:00000210 00000008H .CRT$XPZ                DATA
 0002:00000218 00000008H .CRT$XTA                DATA
 0002:00000220 00000010H .CRT$XTZ                DATA
 0002:00000228 00000000H .gehcont$y              DATA
 0002:00000228 00000000H .gfids$y                DATA
 0002:00000230 00001ed0H .rdata                  DATA
 0002:00002100 00000000H .rdata$CastGuardVftablesA DATA
 0002:00002100 00000000H .rdata$CastGuardVftablesC DATA
 0002:00002100 00000028H .rdata$T                DATA
 0002:00002128 000000a4H .rdata$voltmd           DATA
 0002:000021cc 0000031cH .rdata$zzzdbg           DATA
 0002:000024e8 00000008H .rtc$IAA                DATA
 0002:000024f0 00000008H .rtc$IZZ                DATA
 0002:000024f8 00000008H .rtc$TAA                DATA
 0002:00002500 00000008H .rtc$TZZ                DATA
 0002:00002508 00000004H .tls                    DATA
 0002:0000250c 00000004H .tls$                   DATA
 0002:00002510 00000008H .tls$ZZZ                DATA
 0002:00002518 00000308H .xdata                  DATA
 0002:00002820 000003f4H .edata                  DATA
 0002:00002c14 00000064H .idata$2                DATA
 0002:00002c78 00000018H .idata$3                DATA
 0002:00002c90 00000198H .idata$4                DATA
 0002:00002e28 0000041eH .idata$6                DATA
 0003:00000000 00000090H .data                   DATA
 0003:00000090 0001b248H .bss                    DATA
 0004:00000000 00000384H .pdata                  DATA

  Address         Publics by Value              Rva+Base               Lib:Object

 0000:00000000       __AbsoluteZero             0000000000000000     <absolute>
 0000:00000000       ___safe_se_handler_count   0000000000000000     <absolute>
 0000:00000000       ___safe_se_handler_table   0000000000000000     <absolute>
 0000:00000000       __arm64x_extra_rfe_table   0000000000000000     <absolute>
 0000:00000000       __arm64x_extra_rfe_table_size 0000000000000000     <absolute>
 0000:00000000       __arm64x_native_entrypoint 0000000000000000     <absolute>
 0000:00000000       __arm64x_redirection_metadata 0000000000000000     <absolute>
 0000:00000000       __arm64x_redirection_metadata_count 0000000000000000     <absolute>
 0000:00000000       __dynamic_value_reloc_table 0000000000000000     <absolute>
 0000:00000000       __enclave_config           0000000000000000     <absolute>
 0000:00000000       __guard_check_icall_a64n_fptr 0000000000000000     <absolute>
 0000:00000000       __guard_eh_cont_count      0000000000000000     <absolute>
 0000:00000000       __guard_eh_cont_table      0000000000000000     <absolute>
 0000:00000000       __guard_fids_count         0000000000000000     <absolute>
 0000:00000000       __guard_fids_table         0000000000000000     <absolute>
 0000:00000000       __guard_iat_count          0000000000000000     <absolute>
 0000:00000000       __guard_iat_table          0000000000000000     <absolute>
 0000:00000000       __guard_longjmp_count      0000000000000000     <absolute>
 0000:00000000       __guard_longjmp_table      0000000000000000     <absolute>
 0000:00000000       __hybrid_auxiliary_iat     0000000000000000     <absolute>
 0000:00000000       __hybrid_auxiliary_iat_copy 0000000000000000     <absolute>
 0000:00000000       __hybrid_code_map          0000000000000000     <absolute>
 0000:00000000       __hybrid_code_map_count    0000000000000000     <absolute>
 0000:00000000       __x64_code_ranges_to_entry_points 0000000000000000     <absolute>
 0000:00000000       __x64_code_ranges_to_entry_points_count 0000000000000000     <absolute>
 0000:00000100       __guard_flags              0000000000000100     <absolute>
 0000:00000000       __ImageBase                0000000180000000     <linker-defined>
 0001:00000000       ?NewObject@JNIEnv_@@QEAAPEAV_jobject@@PEAV_jclass@@PEAU_jmethodID@@ZZ 0000000180001000 f i libredefclass004.obj
 0001:00000028       ?TranslateError@@YAPEBDW4jvmtiError@@@Z 0000000180001028 f   libredefclass004.obj
 0001:000002e0       ?nsk_jni_check_exception@@YAHPEAUJNIEnv_@@QEBDH@Z 00000001800012e0 f   libredefclass004.obj
 0001:00000424       ?nsk_jni_lverify@@YAHHPEAUJNIEnv_@@HQEBDH1ZZ 0000000180001424 f   libredefclass004.obj
 0001:000004c4       Agent_Initialize           00000001800014c4 f   libredefclass004.obj
 0001:000005cc       Agent_OnAttach             00000001800015cc f   libredefclass004.obj
 0001:000005cc       Agent_OnLoad               00000001800015cc f   libredefclass004.obj
 0001:000005d4       Java_nsk_jvmti_RedefineClasses_redefclass004_checkNewFields 00000001800015d4 f   libredefclass004.obj
 0001:000007ec       Java_nsk_jvmti_RedefineClasses_redefclass004_makeRedefinition 00000001800017ec f   libredefclass004.obj
 0001:00000910       Java_nsk_jvmti_unit_FollowReferences_FollowRefObjects_addRefToVerify 0000000180001910 f   libredefclass004.obj
 0001:00000ae8       Java_nsk_jvmti_unit_FollowReferences_FollowRefObjects_getTag 0000000180001ae8 f   libredefclass004.obj
 0001:00000ba8       Java_nsk_jvmti_unit_FollowReferences_FollowRefObjects_resetRefsToVerify 0000000180001ba8 f   libredefclass004.obj
 0001:00000bb0       Java_nsk_jvmti_unit_FollowReferences_FollowRefObjects_resetTags 0000000180001bb0 f   libredefclass004.obj
 0001:00000bf4       Java_nsk_jvmti_unit_FollowReferences_FollowRefObjects_setTag 0000000180001bf4 f   libredefclass004.obj
 0001:00000e4c       Java_nsk_share_jvmti_ArgumentHandler_getAgentOptionsString 0000000180001e4c f   libredefclass004.obj
 0001:00000efc       Java_nsk_share_jvmti_DebugeeClass_checkStatus 0000000180001efc f   libredefclass004.obj
 0001:00000f84       Java_nsk_share_jvmti_DebugeeClass_resetAgentData 0000000180001f84 f   libredefclass004.obj
 0001:00000fe4       Java_nsk_share_jvmti_RedefineAgent_agentStatus 0000000180001fe4 f   libredefclass004.obj
 0001:00000ff0       Java_nsk_share_jvmti_RedefineAgent_isRedefined 0000000180001ff0 f   libredefclass004.obj
 0001:00000ffc       Java_nsk_share_jvmti_RedefineAgent_redefineAttempted 0000000180001ffc f   libredefclass004.obj
 0001:00001008       MA_checkStatus             0000000180002008 f   libredefclass004.obj
 0001:000010ac       __local_stdio_printf_options 00000001800020ac f i libredefclass004.obj
 0001:0000128c       exitOnError                000000018000228c f   libredefclass004.obj
 0001:00001340       fprintf                    0000000180002340 f i libredefclass004.obj
 0001:00001384       nsk_jvmti_lverify          0000000180002384 f   libredefclass004.obj
 0001:00001474       nsk_jvmti_resetAgentData   0000000180002474 f   libredefclass004.obj
 0001:000014f4       nsk_jvmti_setFailStatus    00000001800024f4 f   libredefclass004.obj
 0001:00001530       nsk_lcomplain              0000000180002530 f   libredefclass004.obj
 0001:00001550       nsk_ldisplay               0000000180002550 f   libredefclass004.obj
 0001:00001570       nsk_ltrace                 0000000180002570 f   libredefclass004.obj
 0001:00001590       nsk_lvcomplain             0000000180002590 f   libredefclass004.obj
 0001:00001748       nsk_lvdisplay              0000000180002748 f   libredefclass004.obj
 0001:00001794       nsk_lverify                0000000180002794 f   libredefclass004.obj
 0001:000017f0       nsk_lvtrace                00000001800027f0 f   libredefclass004.obj
 0001:00001850       nsk_printf                 0000000180002850 f   libredefclass004.obj
 0001:00001878       nsk_vprintf                0000000180002878 f   libredefclass004.obj
 0001:0000192c       printf                     000000018000292c f i libredefclass004.obj
 0001:00001e54       __raise_securityfailure    0000000180002e54 f   MSVCRT:gs_report.obj
 0001:00001e88       __report_gsfailure         0000000180002e88 f   MSVCRT:gs_report.obj
 0001:000020c8       __GSHandlerCheck           00000001800030c8 f   MSVCRT:gshandler.obj
 0001:000020e8       __GSHandlerCheckCommon     00000001800030e8 f   MSVCRT:gshandler.obj
 0001:00002160       __security_check_cookie    0000000180003160 f   MSVCRT:amdsecgs.obj
 0001:000024a0       _DllMainCRTStartup         00000001800034a0 f   MSVCRT:dll_dllmain.obj
 0001:000024e0       __scrt_acquire_startup_lock 00000001800034e0 f   MSVCRT:utility.obj
 0001:0000251c       __scrt_dllmain_after_initialize_c 000000018000351c f   MSVCRT:utility.obj
 0001:00002550       __scrt_dllmain_before_initialize_c 0000000180003550 f   MSVCRT:utility.obj
 0001:00002568       __scrt_dllmain_crt_thread_attach 0000000180003568 f   MSVCRT:utility.obj
 0001:00002590       __scrt_dllmain_crt_thread_detach 0000000180003590 f   MSVCRT:utility.obj
 0001:000025a8       __scrt_dllmain_exception_filter 00000001800035a8 f   MSVCRT:utility.obj
 0001:00002608       __scrt_dllmain_uninitialize_c 0000000180003608 f   MSVCRT:utility.obj
 0001:00002638       __scrt_dllmain_uninitialize_critical 0000000180003638 f   MSVCRT:utility.obj
 0001:0000264c       __scrt_initialize_crt      000000018000364c f   MSVCRT:utility.obj
 0001:00002698       __scrt_initialize_onexit_tables 0000000180003698 f   MSVCRT:utility.obj
 0001:00002724       __scrt_is_nonwritable_in_current_image 0000000180003724 f   MSVCRT:utility.obj
 0001:000027bc       __scrt_release_startup_lock 00000001800037bc f   MSVCRT:utility.obj
 0001:000027e0       __scrt_uninitialize_crt    00000001800037e0 f   MSVCRT:utility.obj
 0001:0000280c       _onexit                    000000018000380c f   MSVCRT:utility.obj
 0001:00002848       atexit                     0000000180003848 f   MSVCRT:utility.obj
 0001:00002860       __crt_debugger_hook        0000000180003860 f   MSVCRT:utility_desktop.obj
 0001:00002868       __scrt_fastfail            0000000180003868 f   MSVCRT:utility_desktop.obj
 0001:000029b4       _guard_check_icall_nop     00000001800039b4 f i MSVCRT:guard_support.obj
 0001:000029b8       __security_init_cookie     00000001800039b8 f   MSVCRT:gs_support.obj
 0001:00002a64       DllMain                    0000000180003a64 f   MSVCRT:dll_dllmain_stub.obj
 0001:00002a88       ?__scrt_initialize_type_info@@YAXXZ 0000000180003a88 f   MSVCRT:tncleanup.obj
 0001:00002a98       ?__scrt_uninitialize_type_info@@YAXXZ 0000000180003a98 f   MSVCRT:tncleanup.obj
 0001:00002aa4       __local_stdio_scanf_options 0000000180003aa4 f i MSVCRT:default_local_stdio_options.obj
 0001:00002aac       __scrt_initialize_default_local_stdio_options 0000000180003aac f   MSVCRT:default_local_stdio_options.obj
 0001:00002ac8       __scrt_get_dyn_tls_init_callback 0000000180003ac8 f   MSVCRT:dyn_tls_init.obj
 0001:00002ad0       _RTC_Initialize            0000000180003ad0 f   MSVCRT:initsect.obj
 0001:00002b0c       _RTC_Terminate             0000000180003b0c f   MSVCRT:initsect.obj
 0001:00002b48       __isa_available_init       0000000180003b48 f   MSVCRT:cpu_disp.obj
 0001:00002cf4       _get_startup_argv_mode     0000000180003cf4 f   MSVCRT:argv_mode.obj
 0001:00002cfc       __scrt_is_ucrt_dll_in_use  0000000180003cfc f   MSVCRT:ucrt_detection.obj
 0001:00002d10       memcpy                     0000000180003d10 f   vcruntime:VCRUNTIME140.dll
 0001:00002d16       memset                     0000000180003d16 f   vcruntime:VCRUNTIME140.dll
 0001:00002d1c       strchr                     0000000180003d1c f   vcruntime:VCRUNTIME140.dll
 0001:00002d22       __C_specific_handler       0000000180003d22 f   vcruntime:VCRUNTIME140.dll
 0001:00002d28       __std_type_info_destroy_list 0000000180003d28 f   vcruntime:VCRUNTIME140.dll
 0001:00002d2e       strcmp                     0000000180003d2e f   ucrt:api-ms-win-crt-string-l1-1-0.dll
 0001:00002d34       strlen                     0000000180003d34 f   ucrt:api-ms-win-crt-string-l1-1-0.dll
 0001:00002d3a       _initterm                  0000000180003d3a f   ucrt:api-ms-win-crt-runtime-l1-1-0.dll
 0001:00002d40       _initterm_e                0000000180003d40 f   ucrt:api-ms-win-crt-runtime-l1-1-0.dll
 0001:00002d46       _seh_filter_dll            0000000180003d46 f   ucrt:api-ms-win-crt-runtime-l1-1-0.dll
 0001:00002d4c       _configure_narrow_argv     0000000180003d4c f   ucrt:api-ms-win-crt-runtime-l1-1-0.dll
 0001:00002d52       _initialize_narrow_environment 0000000180003d52 f   ucrt:api-ms-win-crt-runtime-l1-1-0.dll
 0001:00002d58       _initialize_onexit_table   0000000180003d58 f   ucrt:api-ms-win-crt-runtime-l1-1-0.dll
 0001:00002d5e       _register_onexit_function  0000000180003d5e f   ucrt:api-ms-win-crt-runtime-l1-1-0.dll
 0001:00002d64       _execute_onexit_table      0000000180003d64 f   ucrt:api-ms-win-crt-runtime-l1-1-0.dll
 0001:00002d6a       _crt_atexit                0000000180003d6a f   ucrt:api-ms-win-crt-runtime-l1-1-0.dll
 0001:00002d70       _cexit                     0000000180003d70 f   ucrt:api-ms-win-crt-runtime-l1-1-0.dll
 0001:00002d78       __acrt_initialize          0000000180003d78 f   MSVCRT:ucrt_stubs.obj
 0001:00002d78       __acrt_thread_attach       0000000180003d78 f   MSVCRT:ucrt_stubs.obj
 0001:00002d78       __acrt_thread_detach       0000000180003d78 f   MSVCRT:ucrt_stubs.obj
 0001:00002d78       __acrt_uninitialize        0000000180003d78 f   MSVCRT:ucrt_stubs.obj
 0001:00002d78       __acrt_uninitialize_critical 0000000180003d78 f   MSVCRT:ucrt_stubs.obj
 0001:00002d78       __scrt_stub_for_acrt_initialize 0000000180003d78 f   MSVCRT:ucrt_stubs.obj
 0001:00002d78       __scrt_stub_for_acrt_thread_attach 0000000180003d78 f   MSVCRT:ucrt_stubs.obj
 0001:00002d78       __scrt_stub_for_acrt_thread_detach 0000000180003d78 f   MSVCRT:ucrt_stubs.obj
 0001:00002d78       __scrt_stub_for_acrt_uninitialize 0000000180003d78 f   MSVCRT:ucrt_stubs.obj
 0001:00002d78       __scrt_stub_for_acrt_uninitialize_critical 0000000180003d78 f   MSVCRT:ucrt_stubs.obj
 0001:00002d78       __vcrt_initialize          0000000180003d78 f   MSVCRT:ucrt_stubs.obj
 0001:00002d78       __vcrt_thread_attach       0000000180003d78 f   MSVCRT:ucrt_stubs.obj
 0001:00002d78       __vcrt_thread_detach       0000000180003d78 f   MSVCRT:ucrt_stubs.obj
 0001:00002d78       __vcrt_uninitialize        0000000180003d78 f   MSVCRT:ucrt_stubs.obj
 0001:00002d78       __vcrt_uninitialize_critical 0000000180003d78 f   MSVCRT:ucrt_stubs.obj
 0001:00002d7c       __scrt_stub_for_is_c_termination_complete 0000000180003d7c f   MSVCRT:ucrt_stubs.obj
 0001:00002d7c       _is_c_termination_complete 0000000180003d7c f   MSVCRT:ucrt_stubs.obj
 0001:00002d90       _guard_dispatch_icall_nop  0000000180003d90 f   MSVCRT:guard_dispatch.obj
 0001:00002db0       _guard_xfg_dispatch_icall_nop 0000000180003db0 f   MSVCRT:guard_xfg_dispatch.obj
 0002:00000000       __imp_RtlCaptureContext    0000000180004000     kernel32:KERNEL32.dll
 0002:00000008       __imp_RtlLookupFunctionEntry 0000000180004008     kernel32:KERNEL32.dll
 0002:00000010       __imp_RtlVirtualUnwind     0000000180004010     kernel32:KERNEL32.dll
 0002:00000018       __imp_UnhandledExceptionFilter 0000000180004018     kernel32:KERNEL32.dll
 0002:00000020       __imp_SetUnhandledExceptionFilter 0000000180004020     kernel32:KERNEL32.dll
 0002:00000028       __imp_GetCurrentProcess    0000000180004028     kernel32:KERNEL32.dll
 0002:00000030       __imp_TerminateProcess     0000000180004030     kernel32:KERNEL32.dll
 0002:00000038       __imp_IsProcessorFeaturePresent 0000000180004038     kernel32:KERNEL32.dll
 0002:00000040       __imp_CloseHandle          0000000180004040     kernel32:KERNEL32.dll
 0002:00000048       __imp_InitializeCriticalSectionAndSpinCount 0000000180004048     kernel32:KERNEL32.dll
 0002:00000050       __imp_DeleteCriticalSection 0000000180004050     kernel32:KERNEL32.dll
 0002:00000058       __imp_CreateEventW         0000000180004058     kernel32:KERNEL32.dll
 0002:00000060       __imp_GetModuleHandleW     0000000180004060     kernel32:KERNEL32.dll
 0002:00000068       __imp_GetProcAddress       0000000180004068     kernel32:KERNEL32.dll
 0002:00000070       __imp_IsDebuggerPresent    0000000180004070     kernel32:KERNEL32.dll
 0002:00000078       __imp_QueryPerformanceCounter 0000000180004078     kernel32:KERNEL32.dll
 0002:00000080       __imp_GetCurrentProcessId  0000000180004080     kernel32:KERNEL32.dll
 0002:00000088       __imp_GetCurrentThreadId   0000000180004088     kernel32:KERNEL32.dll
 0002:00000090       __imp_GetSystemTimeAsFileTime 0000000180004090     kernel32:KERNEL32.dll
 0002:00000098       __imp_DisableThreadLibraryCalls 0000000180004098     kernel32:KERNEL32.dll
 0002:000000a0       __imp_InitializeSListHead  00000001800040a0     kernel32:KERNEL32.dll
 0002:000000a8       \177KERNEL32_NULL_THUNK_DATA 00000001800040a8     kernel32:KERNEL32.dll
 0002:000000b0       __imp_memcpy               00000001800040b0     vcruntime:VCRUNTIME140.dll
 0002:000000b8       __imp_memset               00000001800040b8     vcruntime:VCRUNTIME140.dll
 0002:000000c0       __imp_strchr               00000001800040c0     vcruntime:VCRUNTIME140.dll
 0002:000000c8       __imp___C_specific_handler 00000001800040c8     vcruntime:VCRUNTIME140.dll
 0002:000000d0       __imp___std_type_info_destroy_list 00000001800040d0     vcruntime:VCRUNTIME140.dll
 0002:000000d8       \177VCRUNTIME140_NULL_THUNK_DATA 00000001800040d8     vcruntime:VCRUNTIME140.dll
 0002:000000e0       __imp__errno               00000001800040e0     ucrt:api-ms-win-crt-runtime-l1-1-0.dll
 0002:000000e8       __imp_exit                 00000001800040e8     ucrt:api-ms-win-crt-runtime-l1-1-0.dll
 0002:000000f0       __imp__cexit               00000001800040f0     ucrt:api-ms-win-crt-runtime-l1-1-0.dll
 0002:000000f8       __imp__crt_atexit          00000001800040f8     ucrt:api-ms-win-crt-runtime-l1-1-0.dll
 0002:00000100       __imp__execute_onexit_table 0000000180004100     ucrt:api-ms-win-crt-runtime-l1-1-0.dll
 0002:00000108       __imp__register_onexit_function 0000000180004108     ucrt:api-ms-win-crt-runtime-l1-1-0.dll
 0002:00000110       __imp__initialize_onexit_table 0000000180004110     ucrt:api-ms-win-crt-runtime-l1-1-0.dll
 0002:00000118       __imp__initialize_narrow_environment 0000000180004118     ucrt:api-ms-win-crt-runtime-l1-1-0.dll
 0002:00000120       __imp__configure_narrow_argv 0000000180004120     ucrt:api-ms-win-crt-runtime-l1-1-0.dll
 0002:00000128       __imp__seh_filter_dll      0000000180004128     ucrt:api-ms-win-crt-runtime-l1-1-0.dll
 0002:00000130       __imp__initterm_e          0000000180004130     ucrt:api-ms-win-crt-runtime-l1-1-0.dll
 0002:00000138       __imp__initterm            0000000180004138     ucrt:api-ms-win-crt-runtime-l1-1-0.dll
 0002:00000140       \177api-ms-win-crt-runtime-l1-1-0_NULL_THUNK_DATA 0000000180004140     ucrt:api-ms-win-crt-runtime-l1-1-0.dll
 0002:00000148       __imp___acrt_iob_func      0000000180004148     ucrt:api-ms-win-crt-stdio-l1-1-0.dll
 0002:00000150       __imp_fflush               0000000180004150     ucrt:api-ms-win-crt-stdio-l1-1-0.dll
 0002:00000158       __imp___stdio_common_vsprintf 0000000180004158     ucrt:api-ms-win-crt-stdio-l1-1-0.dll
 0002:00000160       __imp___stdio_common_vfprintf 0000000180004160     ucrt:api-ms-win-crt-stdio-l1-1-0.dll
 0002:00000168       \177api-ms-win-crt-stdio-l1-1-0_NULL_THUNK_DATA 0000000180004168     ucrt:api-ms-win-crt-stdio-l1-1-0.dll
 0002:00000170       __imp_strcmp               0000000180004170     ucrt:api-ms-win-crt-string-l1-1-0.dll
 0002:00000178       __imp__strdup              0000000180004178     ucrt:api-ms-win-crt-string-l1-1-0.dll
 0002:00000178       __imp_strdup               0000000180004178     ucrt:api-ms-win-crt-string-l1-1-0.dll
 0002:00000180       __imp_strlen               0000000180004180     ucrt:api-ms-win-crt-string-l1-1-0.dll
 0002:00000188       __imp_strncpy              0000000180004188     ucrt:api-ms-win-crt-string-l1-1-0.dll
 0002:00000190       \177api-ms-win-crt-string-l1-1-0_NULL_THUNK_DATA 0000000180004190     ucrt:api-ms-win-crt-string-l1-1-0.dll
 0002:00000198       __guard_check_icall_fptr   0000000180004198     MSVCRT:guard_support.obj
 0002:000001a0       __guard_xfg_check_icall_fptr 00000001800041a0     MSVCRT:guard_support.obj
 0002:000001a8       __guard_dispatch_icall_fptr 00000001800041a8     MSVCRT:guard_support.obj
 0002:000001b0       __guard_xfg_dispatch_icall_fptr 00000001800041b0     MSVCRT:guard_support.obj
 0002:000001b8       __guard_xfg_table_dispatch_icall_fptr 00000001800041b8     MSVCRT:guard_support.obj
 0002:000001c0       __castguard_check_failure_os_handled_fptr 00000001800041c0     MSVCRT:guard_support.obj
 0002:000001c8       __guard_memcpy_fptr        00000001800041c8     vcruntime:softmemtag.obj
 0002:000001d0       __xc_a                     00000001800041d0     MSVCRT:initializers.obj
 0002:000001d8       __xc_z                     00000001800041d8     MSVCRT:initializers.obj
 0002:000001e0       __xi_a                     00000001800041e0     MSVCRT:initializers.obj
 0002:000001f0       __xi_z                     00000001800041f0     MSVCRT:initializers.obj
 0002:000001f8       __xl_a                     00000001800041f8     MSVCRT:tlssup.obj
 0002:00000200       __xl_z                     0000000180004200     MSVCRT:tlssup.obj
 0002:00000208       __xp_a                     0000000180004208     MSVCRT:initializers.obj
 0002:00000210       __xp_z                     0000000180004210     MSVCRT:initializers.obj
 0002:00000218       __xt_a                     0000000180004218     MSVCRT:initializers.obj
 0002:00000220       __xt_z                     0000000180004220     MSVCRT:initializers.obj
 0002:00000230       g_refKindStr               0000000180004230     libredefclass004.obj
 0002:000003e0       ??_C@_09BPLDFGCI@unknown_0@ 00000001800043e0     libredefclass004.obj
 0002:000003f0       ??_C@_0BL@FPNMECJD@JVMTI_HEAP_REFERENCE_CLASS@ 00000001800043f0     libredefclass004.obj
 0002:00000410       ??_C@_0BL@FKGKKLNM@JVMTI_HEAP_REFERENCE_FIELD@ 0000000180004410     libredefclass004.obj
 0002:00000430       ??_C@_0CD@CAEHCFJF@JVMTI_HEAP_REFERENCE_ARRAY_ELEM@ 0000000180004430     libredefclass004.obj
 0002:00000458       ??_C@_0CC@DNEBMCNK@JVMTI_HEAP_REFERENCE_CLASS_LOAD@ 0000000180004458     libredefclass004.obj
 0002:00000480       ??_C@_0BN@CJMIPEBB@JVMTI_HEAP_REFERENCE_SIGNERS@ 0000000180004480     libredefclass004.obj
 0002:000004a0       ??_C@_0CH@HBOIDPEB@JVMTI_HEAP_REFERENCE_PROTECTION@ 00000001800044a0     libredefclass004.obj
 0002:000004c8       ??_C@_0BP@MDKGDGKL@JVMTI_HEAP_REFERENCE_INTERFACE@ 00000001800044c8     libredefclass004.obj
 0002:000004e8       ??_C@_0CC@JJMIHNJH@JVMTI_HEAP_REFERENCE_STATIC_FIE@ 00000001800044e8     libredefclass004.obj
 0002:00000510       ??_C@_0CD@IDHEEGID@JVMTI_HEAP_REFERENCE_CONSTANT_P@ 0000000180004510     libredefclass004.obj
 0002:00000538       ??_C@_0CA@EFFCHNG@JVMTI_HEAP_REFERENCE_SUPERCLASS@ 0000000180004538     libredefclass004.obj
 0002:00000558       ??_C@_0L@PCDFHGCJ@unknown_11@ 0000000180004558     libredefclass004.obj
 0002:00000568       ??_C@_0L@NJBICFOK@unknown_12@ 0000000180004568     libredefclass004.obj
 0002:00000578       ??_C@_0L@MAADBEKL@unknown_13@ 0000000180004578     libredefclass004.obj
 0002:00000588       ??_C@_0L@IPECICGM@unknown_14@ 0000000180004588     libredefclass004.obj
 0002:00000598       ??_C@_0L@JGFJLDCN@unknown_15@ 0000000180004598     libredefclass004.obj
 0002:000005a8       ??_C@_0L@LNHEOAOO@unknown_16@ 00000001800045a8     libredefclass004.obj
 0002:000005b8       ??_C@_0L@KEGPNBKP@unknown_17@ 00000001800045b8     libredefclass004.obj
 0002:000005c8       ??_C@_0L@CDPHMNGA@unknown_18@ 00000001800045c8     libredefclass004.obj
 0002:000005d8       ??_C@_0L@DKOMPMCB@unknown_19@ 00000001800045d8     libredefclass004.obj
 0002:000005e8       ??_C@_0L@OJGIPJDB@unknown_20@ 00000001800045e8     libredefclass004.obj
 0002:000005f8       ??_C@_0CA@KAOFNDEM@JVMTI_HEAP_REFERENCE_JNI_GLOBAL@ 00000001800045f8     libredefclass004.obj
 0002:00000618       ??_C@_0CC@HPFAJBK@JVMTI_HEAP_REFERENCE_SYSTEM_CLA@ 0000000180004618     libredefclass004.obj
 0002:00000640       ??_C@_0BN@FDEGFOHC@JVMTI_HEAP_REFERENCE_MONITOR@ 0000000180004640     libredefclass004.obj
 0002:00000660       ??_C@_0CB@HKIBCMAJ@JVMTI_HEAP_REFERENCE_STACK_LOCA@ 0000000180004660     libredefclass004.obj
 0002:00000688       ??_C@_0BP@EAACMMOE@JVMTI_HEAP_REFERENCE_JNI_LOCAL@ 0000000180004688     libredefclass004.obj
 0002:000006a8       ??_C@_0BM@IJDEOGOE@JVMTI_HEAP_REFERENCE_THREAD@ 00000001800046a8     libredefclass004.obj
 0002:000006c8       ??_C@_0BL@EDGPPKC@JVMTI_HEAP_REFERENCE_OTHER@ 00000001800046c8     libredefclass004.obj
 0002:000006e4       ??_C@_04BCJPDBDA@Code@     00000001800046e4     libredefclass004.obj
 0002:000006f0       ??_C@_0BA@OCLMCFKC@LineNumberTable@ 00000001800046f0     libredefclass004.obj
 0002:00000700       ??_C@_0BD@CPAEPILC@LocalVariableTable@ 0000000180004700     libredefclass004.obj
 0002:00000718       ??_C@_0BH@NMBDNHBD@LocalVariableTypeTable@ 0000000180004718     libredefclass004.obj
 0002:00000730       ??_C@_0O@HIHEEDNJ@StackMapTable@ 0000000180004730     libredefclass004.obj
 0002:00000740       ??_C@_0L@HCDIAMJG@?9?5?$CFs?0?5?$CFd?3?5@ 0000000180004740     libredefclass004.obj
 0002:00000750       ??_C@_0JI@HLPECLFI@?$CD?5?4?4?4?6?$CD?5ERROR?3?5too?5many?5complai@ 0000000180004750     libredefclass004.obj
 0002:000007f0       ??_C@_0ED@JNEKCCOB@The?5following?5fake?5exception?5st@ 00000001800047f0     libredefclass004.obj
 0002:00000838       ??_C@_0CN@FCNMDFBH@nsk?4share?4Fake_Exception_for_RU@ 0000000180004838     libredefclass004.obj
 0002:00000868       ??_C@_08PGFFNAEI@?$CI?$CFs?3?$CFd?$CJ?5@ 0000000180004868     libredefclass004.obj
 0002:00000878       ??_C@_0DP@IENMAEGI@s?2test?2hotspot?2jtreg?2vmTestbase@ 0000000180004878     libredefclass004.obj
 0002:000008b8       ??_C@_0BL@NDJLFFJB@?7at?5nsk_lvcomplain?$CI?$CFs?3?$CFd?$CJ?6@ 00000001800048b8     libredefclass004.obj
 0002:000008d8       ??_C@_0BC@JOOKAFKF@?$CD?5ERROR?3?5?$CFs?0?5?$CFd?3?5@ 00000001800048d8     libredefclass004.obj
 0002:000008f0       ??_C@_09KJEAHMEH@?$CD?5ERROR?3?5@ 00000001800048f0     libredefclass004.obj
 0002:000008fc       ??_C@_02GPIOPFAK@?$DO?$DO@ 00000001800048fc     libredefclass004.obj
 0002:00000900       ??_C@_02FODMEDOG@?$DM?$DM@ 0000000180004900     libredefclass004.obj
 0002:00000904       ??_C@_02DJGKEECL@?4?4@     0000000180004904     libredefclass004.obj
 0002:00000908       ??_C@_0O@CJPGJOAF@?9?5?$CFs?0?5?$CFd?3?5?$CFs?5@ 0000000180004908     libredefclass004.obj
 0002:00000918       ??_C@_0CB@IAKPDOIC@?$CD?5?5?5verified?5assertion?5is?5FALSE@ 0000000180004918     libredefclass004.obj
 0002:00000940       ??_C@_0CO@LGONDEPD@stdout?3?5fflush?5failed?5?9?5err?$DN?$CFd?5@ 0000000180004940     libredefclass004.obj
 0002:00000970       ??_C@_0CO@KBGKJPBD@stderr?3?5fflush?5failed?5?9?5err?$DN?$CFd?5@ 0000000180004970     libredefclass004.obj
 0002:000009a0       ??_C@_0BB@JCNMKLLK@JVMTI_ERROR_NONE@ 00000001800049a0     libredefclass004.obj
 0002:000009b8       ??_C@_0BL@LDIMKLPH@JVMTI_ERROR_INVALID_THREAD@ 00000001800049b8     libredefclass004.obj
 0002:000009d8       ??_C@_0CB@PJFPAIKJ@JVMTI_ERROR_INVALID_THREAD_GROU@ 00000001800049d8     libredefclass004.obj
 0002:00000a00       ??_C@_0BN@LLMKHMNF@JVMTI_ERROR_INVALID_PRIORITY@ 0000000180004a00     libredefclass004.obj
 0002:00000a20       ??_C@_0CB@MBOFKAGB@JVMTI_ERROR_THREAD_NOT_SUSPENDE@ 0000000180004a20     libredefclass004.obj
 0002:00000a48       ??_C@_0BN@FABOLPBI@JVMTI_ERROR_THREAD_SUSPENDED@ 0000000180004a48     libredefclass004.obj
 0002:00000a68       ??_C@_0BN@FDGNOBJM@JVMTI_ERROR_THREAD_NOT_ALIVE@ 0000000180004a68     libredefclass004.obj
 0002:00000a88       ??_C@_0BL@GOBIFKNJ@JVMTI_ERROR_INVALID_OBJECT@ 0000000180004a88     libredefclass004.obj
 0002:00000aa8       ??_C@_0BK@FCMAJPPC@JVMTI_ERROR_INVALID_CLASS@ 0000000180004aa8     libredefclass004.obj
 0002:00000ac8       ??_C@_0BP@IKLLBKEB@JVMTI_ERROR_CLASS_NOT_PREPARED@ 0000000180004ac8     libredefclass004.obj
 0002:00000ae8       ??_C@_0BN@KLPPLKG@JVMTI_ERROR_INVALID_METHODID@ 0000000180004ae8     libredefclass004.obj
 0002:00000b08       ??_C@_0BN@BCEKOKND@JVMTI_ERROR_INVALID_LOCATION@ 0000000180004b08     libredefclass004.obj
 0002:00000b28       ??_C@_0BM@DFDGPME@JVMTI_ERROR_INVALID_FIELDID@ 0000000180004b28     libredefclass004.obj
 0002:00000b48       ??_C@_0BL@NELIEPEC@JVMTI_ERROR_NO_MORE_FRAMES@ 0000000180004b48     libredefclass004.obj
 0002:00000b68       ??_C@_0BJ@BDBECFDM@JVMTI_ERROR_OPAQUE_FRAME@ 0000000180004b68     libredefclass004.obj
 0002:00000b88       ??_C@_0BK@MIIFNLOB@JVMTI_ERROR_TYPE_MISMATCH@ 0000000180004b88     libredefclass004.obj
 0002:00000ba8       ??_C@_0BJ@HPCAOILC@JVMTI_ERROR_INVALID_SLOT@ 0000000180004ba8     libredefclass004.obj
 0002:00000bc8       ??_C@_0BG@CHILOPNI@JVMTI_ERROR_DUPLICATE@ 0000000180004bc8     libredefclass004.obj
 0002:00000be0       ??_C@_0BG@DIEMLHKM@JVMTI_ERROR_NOT_FOUND@ 0000000180004be0     libredefclass004.obj
 0002:00000bf8       ??_C@_0BM@NHMCKHOB@JVMTI_ERROR_INVALID_MONITOR@ 0000000180004bf8     libredefclass004.obj
 0002:00000c18       ??_C@_0BO@PPEDAJGL@JVMTI_ERROR_NOT_MONITOR_OWNER@ 0000000180004c18     libredefclass004.obj
 0002:00000c38       ??_C@_0BG@FCAIPEID@JVMTI_ERROR_INTERRUPT@ 0000000180004c38     libredefclass004.obj
 0002:00000c50       ??_C@_0CB@EGDBNKOI@JVMTI_ERROR_INVALID_CLASS_FORMA@ 0000000180004c50     libredefclass004.obj
 0002:00000c78       ??_C@_0CG@DGKOGIAL@JVMTI_ERROR_CIRCULAR_CLASS_DEFI@ 0000000180004c78     libredefclass004.obj
 0002:00000ca0       ??_C@_0BP@ICEALPKC@JVMTI_ERROR_FAILS_VERIFICATION@ 0000000180004ca0     libredefclass004.obj
 0002:00000cc0       ??_C@_0DC@JDACLMIO@JVMTI_ERROR_UNSUPPORTED_REDEFIN@ 0000000180004cc0     libredefclass004.obj
 0002:00000cf8       ??_C@_0DE@GKDKNOMJ@JVMTI_ERROR_UNSUPPORTED_REDEFIN@ 0000000180004cf8     libredefclass004.obj
 0002:00000d30       ??_C@_0BO@LAFKIOG@JVMTI_ERROR_INVALID_TYPESTATE@ 0000000180004d30     libredefclass004.obj
 0002:00000d50       ??_C@_0DH@INDGCLLB@JVMTI_ERROR_UNSUPPORTED_REDEFIN@ 0000000180004d50     libredefclass004.obj
 0002:00000d88       ??_C@_0DE@NHEOMMGI@JVMTI_ERROR_UNSUPPORTED_REDEFIN@ 0000000180004d88     libredefclass004.obj
 0002:00000dc0       ??_C@_0CA@EKPNJOEP@JVMTI_ERROR_UNSUPPORTED_VERSION@ 0000000180004dc0     libredefclass004.obj
 0002:00000de0       ??_C@_0BN@OFFMAHHL@JVMTI_ERROR_NAMES_DONT_MATCH@ 0000000180004de0     libredefclass004.obj
 0002:00000e00       ??_C@_0DN@HHBBLAKE@JVMTI_ERROR_UNSUPPORTED_REDEFIN@ 0000000180004e00     libredefclass004.obj
 0002:00000e40       ??_C@_0DO@HMBGBGNA@JVMTI_ERROR_UNSUPPORTED_REDEFIN@ 0000000180004e40     libredefclass004.obj
 0002:00000e80       ??_C@_0BP@PBECGKHJ@JVMTI_ERROR_UNMODIFIABLE_CLASS@ 0000000180004e80     libredefclass004.obj
 0002:00000ea0       ??_C@_0BK@CANILEHF@JVMTI_ERROR_NOT_AVAILABLE@ 0000000180004ea0     libredefclass004.obj
 0002:00000ec0       ??_C@_0CE@INJKMEFK@JVMTI_ERROR_MUST_POSSESS_CAPABI@ 0000000180004ec0     libredefclass004.obj
 0002:00000ee8       ??_C@_0BJ@LBFPFPDM@JVMTI_ERROR_NULL_POINTER@ 0000000180004ee8     libredefclass004.obj
 0002:00000f08       ??_C@_0BP@CHJPNNEM@JVMTI_ERROR_ABSENT_INFORMATION@ 0000000180004f08     libredefclass004.obj
 0002:00000f28       ??_C@_0BP@OMFMNLC@JVMTI_ERROR_INVALID_EVENT_TYPE@ 0000000180004f28     libredefclass004.obj
 0002:00000f48       ??_C@_0BN@BIBNPHHO@JVMTI_ERROR_ILLEGAL_ARGUMENT@ 0000000180004f48     libredefclass004.obj
 0002:00000f68       ??_C@_0BK@KKNDHDCE@JVMTI_ERROR_NATIVE_METHOD@ 0000000180004f68     libredefclass004.obj
 0002:00000f88       ??_C@_0BK@PMKCFHAE@JVMTI_ERROR_OUT_OF_MEMORY@ 0000000180004f88     libredefclass004.obj
 0002:00000fa8       ??_C@_0BK@NNJBDMNB@JVMTI_ERROR_ACCESS_DENIED@ 0000000180004fa8     libredefclass004.obj
 0002:00000fc8       ??_C@_0BI@GHECLMNC@JVMTI_ERROR_WRONG_PHASE@ 0000000180004fc8     libredefclass004.obj
 0002:00000fe0       ??_C@_0BF@OLIHJOII@JVMTI_ERROR_INTERNAL@ 0000000180004fe0     libredefclass004.obj
 0002:00000ff8       ??_C@_0BO@EOHGKJHI@JVMTI_ERROR_UNATTACHED_THREAD@ 0000000180004ff8     libredefclass004.obj
 0002:00001018       ??_C@_0CA@LKHFDACL@JVMTI_ERROR_INVALID_ENVIRONMENT@ 0000000180005018     libredefclass004.obj
 0002:00001038       ??_C@_0BA@MMFHLOKK@?$DMunknown?5error?$DO@ 0000000180005038     libredefclass004.obj
 0002:00001048       ??_C@_0CF@CBHOKDB@throwable?5?$DN?5jni?9?$DOExceptionOccur@ 0000000180005048     libredefclass004.obj
 0002:00001070       ??_C@_03OFAPEBGM@?$CFs?6@  0000000180005070     libredefclass004.obj
 0002:00001078       ??_C@_0DM@LPIGEGNJ@s?2test?2hotspot?2jtreg?2vmTestbase@ 0000000180005078     libredefclass004.obj
 0002:000010b8       ??_C@_0CC@NFCNPEPK@Exception?5in?5JNI?5call?5?$CIcleared?$CJ@ 00000001800050b8     libredefclass004.obj
 0002:000010e0       ??_C@_0BJ@IBAKFIKF@jni?9?$DOExceptionDescribe?$CI?$CJ@ 00000001800050e0     libredefclass004.obj
 0002:00001100       ??_C@_0BG@GGKALKMH@jni?9?$DOExceptionClear?$CI?$CJ@ 0000000180005100     libredefclass004.obj
 0002:00001118       ??_C@_0CF@JMGFGJLJ@?$CD?5?5?5verified?5JNI?5assertion?5is?5F@ 0000000180005118     libredefclass004.obj
 0002:00001140       ??_C@_0CB@MLNJNCLJ@?5?5jvmti?5error?3?5code?$DN?$CFd?0?5name?$DN?$CFs@ 0000000180005140     libredefclass004.obj
 0002:00001168       ??_C@_0CD@OHBGDKMK@?$CD?5?5?5jvmti?5error?3?5code?$DN?$CFd?0?5name?$DN@ 0000000180005168     libredefclass004.obj
 0002:00001190       ??_C@_0CG@JNNCGPHB@?$CD?5?5?5error?5expected?3?5code?$DN?$CFd?0?5na@ 0000000180005190     libredefclass004.obj
 0002:000011c0       ??_C@_0EB@IMGKPCGE@?$CIstr_obj?5?$DN?5jni?9?$DONewStringUTF?$CIco@ 00000001800051c0     libredefclass004.obj
 0002:00001210       ??_C@_0EA@HFOGGBCC@s?2test?2hotspot?2jtreg?2vmTestbase@ 0000000180005210     libredefclass004.obj
 0002:00001250       ??_C@_05KKCIMGE@error@     0000000180005250     libredefclass004.obj
 0002:00001258       ??_C@_0CJ@JACLEAA@Test?5failed?5by?5setFailStatus?$CI?$CJ?4@ 0000000180005258     libredefclass004.obj
 0002:00001290       ??_C@_0EA@PNBCDMOA@s?2test?2hotspot?2jtreg?2vmTestbase@ 0000000180005290     libredefclass004.obj
 0002:000012d0       ??_C@_0DI@ILAHDLMP@?$CI?$CKagentThreadProc?$CJ?$CIjvmti_env?0?5a@ 00000001800052d0     libredefclass004.obj
 0002:00001308       ??_C@_0BD@KDBALNLB@JVMTI?5agent?5thread@ 0000000180005308     libredefclass004.obj
 0002:00001320       ??_C@_0BB@NOKBFPFO@java?1lang?1Thread@ 0000000180005320     libredefclass004.obj
 0002:00001334       ??_C@_06FALKBLGB@?$DMinit?$DO@ 0000000180005334     libredefclass004.obj
 0002:00001340       ??_C@_0BG@IKDDPPGD@?$CILjava?1lang?1String?$DL?$CJV@ 0000000180005340     libredefclass004.obj
 0002:00001360       ??_C@_0EB@IFJBFEKC@?$CIthreadClass?5?$DN?5jni_env?9?$DOFindCla@ 0000000180005360     libredefclass004.obj
 0002:000013b0       ??_C@_0GF@FGFIBKKL@?$CIthreadCtor?5?$DN?5jni_env?9?$DOGetMetho@ 00000001800053b0     libredefclass004.obj
 0002:00001418       ??_C@_0DN@NCPDJLOG@?$CIthreadName?5?$DN?5jni_env?9?$DONewStrin@ 0000000180005418     libredefclass004.obj
 0002:00001460       ??_C@_0FE@PFKODBGC@?$CIthreadObject?5?$DN?5jni_env?9?$DONewObj@ 0000000180005460     libredefclass004.obj
 0002:000014c0       ??_C@_0ED@HOBAHHJI@?$CIthreadGlobalRef?5?$DN?5jni_env?9?$DONew@ 00000001800054c0     libredefclass004.obj
 0002:00001510       ??_C@_0FN@HNJJAHFC@jvmti_env?9?$DORunAgentThread?$CIagent@ 0000000180005510     libredefclass004.obj
 0002:00001570       ??_C@_0EA@MOJDNKDF@Debuggee?5status?5sync?5aborted?5be@ 0000000180005570     libredefclass004.obj
 0002:000015b0       ??_C@_0EA@EEOEJAEN@status?5?$DN?5syncDebuggeeStatus?$CIjni@ 00000001800055b0     libredefclass004.obj
 0002:000015f0       ??_C@_0BL@JBCFNBMB@nsk_jvmti_resetAgentData?$CI?$CJ@ 00000001800055f0     libredefclass004.obj
 0002:00001610       ??_C@_0EL@LPBEELIP@s?2test?2hotspot?2jtreg?2vmTestbase@ 0000000180005610     libredefclass004.obj
 0002:00001660       ??_C@_0CK@JDAMFDMJ@jvmti?9?$DOSetTag?$CIo?0?5tag?$CJ?5?$DN?$DN?5JVMTI_@ 0000000180005660     libredefclass004.obj
 0002:00001690       ??_C@_0CC@DAMNHKNI@Can?8t?5set?5tag?5?$CFli?5for?5object?5?$CFl@ 0000000180005690     libredefclass004.obj
 0002:000016b8       ??_C@_0DL@HAJPNKEF@jvmti?9?$DOGetObjectHashCode?$CIo?0?5?$CGha@ 00000001800056b8     libredefclass004.obj
 0002:000016f8       ??_C@_0BL@JFPIEOBF@Can?8t?5get?5hash?5object?5?$CFlx?6@ 00000001800056f8     libredefclass004.obj
 0002:00001718       ??_C@_0BG@DICPHBKN@setTag?3?5?$CF08x?5?$DM?9?5?$CF?53li@ 0000000180005718     libredefclass004.obj
 0002:00001730       ??_C@_0DH@FCEEBDMJ@?$CIs?5?$DN?5jni?9?$DOGetStringUTFChars?$CIsIn@ 0000000180005730     libredefclass004.obj
 0002:00001768       ??_C@_0BJ@OKKGHDCN@Can?8t?5get?5string?5at?5?$CF?$CDp?6@ 0000000180005768     libredefclass004.obj
 0002:00001788       ??_C@_0BP@EKFLGGFJ@Can?8t?5get?5string?5at?5?$CF?$CDp?3?5null?6@ 0000000180005788     libredefclass004.obj
 0002:000017a8       ??_C@_06ICODBHCL@?5?1?1?5?$CFs@ 00000001800057a8     libredefclass004.obj
 0002:000017b0       ??_C@_0DB@KGFPLEGO@?$CIr?5?$DN?5jvmti?9?$DOGetTag?$CIo?0?5?$CGtag?$CJ?$CJ?5?$DN?$DN@ 00000001800057b0     libredefclass004.obj
 0002:000017e8       ??_C@_0CO@PDAGBCGJ@Can?8t?5GetTag?5for?5object?5?$CFlx?4?5Re@ 00000001800057e8     libredefclass004.obj
 0002:00001818       ??_C@_0CH@HPEODOHC@TEST_BUG?3?5Max?4?5number?5of?5refs?5r@ 0000000180005818     libredefclass004.obj
 0002:00001840       ??_C@_0DI@PHFCABIM@?$CIr?5?$DN?5jvmti?9?$DOGetTag?$CIfrom?0?5?$CGtagFr@ 0000000180005840     libredefclass004.obj
 0002:00001878       ??_C@_0DI@MDEGFNKD@TEST_BUG?3?5Can?8t?5GetTag?5for?5obje@ 0000000180005878     libredefclass004.obj
 0002:000018b0       ??_C@_0DE@MLELJAHM@?$CIr?5?$DN?5jvmti?9?$DOGetTag?$CIto?0?5?$CGtagTo?$CJ?$CJ@ 00000001800058b0     libredefclass004.obj
 0002:000018f0       ??_C@_0FK@LMLLKBMP@s?2test?2hotspot?2jtreg?2vmTestbase@ 00000001800058f0     libredefclass004.obj
 0002:00001950       ??_C@_0CF@JMMADLFE@?$CFs?3?5Failed?5to?5call?5GetEnv?3?5erro@ 0000000180005950     libredefclass004.obj
 0002:00001978       ??_C@_0DG@LAJPGIIE@?$CIGetPotentialCapabilities?$CJ?5unex@ 0000000180005978     libredefclass004.obj
 0002:000019b0       ??_C@_0CN@LKPEOJPO@?$CIAddCapabilities?$CJ?5unexpected?5er@ 00000001800059b0     libredefclass004.obj
 0002:000019e0       ??_C@_0CN@BCCBOHCH@?$CIGetCapabilities?$CJ?5unexpected?5er@ 00000001800059e0     libredefclass004.obj
 0002:00001a10       ??_C@_0CN@DLBMMHNI@Warning?3?5RedefineClasses?5is?5not@ 0000000180005a10     libredefclass004.obj
 0002:00001a40       ??_C@_0CH@CDOJMNAO@JVMTI?5client?5was?5not?5properly?5l@ 0000000180005a40     libredefclass004.obj
 0002:00001a68       ??_C@_0DN@HPFPLBDL@?$DO?$DO?$DO?$DO?$DO?$DO?$DO?$DO?5Invoke?5RedefineClasses@ 0000000180005a68     libredefclass004.obj
 0002:00001ab0       ??_C@_0GC@DPGKDDOP@Warning?3?5unrestrictedly?5redefin@ 0000000180005ab0     libredefclass004.obj
 0002:00001b20       ??_C@_0EL@FHLGJEBB@?$CFs?3?5Failed?5to?5call?5RedefineClas@ 0000000180005b20     libredefclass004.obj
 0002:00001b70       ??_C@_0DF@KIBMOCOK@?7For?5more?5info?5about?5this?5error@ 0000000180005b70     libredefclass004.obj
 0002:00001ba8       ??_C@_0DB@JBFCAFBM@?$DM?$DM?$DM?$DM?$DM?$DM?$DM?$DM?5RedefineClasses?$CI?$CJ?5is?5s@ 0000000180005ba8     libredefclass004.obj
 0002:00001bdc       ??_C@_01JPJNBJEM@I@        0000000180005bdc     libredefclass004.obj
 0002:00001be0       ??_C@_0P@PJIKLCE@intComplNewFld@ 0000000180005be0     libredefclass004.obj
 0002:00001bf0       ??_C@_0DP@CEHCMKKB@?$CFs?3?5Failed?5to?5get?5the?5field?5ID?5@ 0000000180005bf0     libredefclass004.obj
 0002:00001c30       ??_C@_01LELAEKIP@J@        0000000180005c30     libredefclass004.obj
 0002:00001c38       ??_C@_0BA@IBKEKDDP@longComplNewFld@ 0000000180005c38     libredefclass004.obj
 0002:00001c50       ??_C@_0EA@PMBNLAHO@?$CFs?3?5Failed?5to?5get?5the?5field?5ID?5@ 0000000180005c50     libredefclass004.obj
 0002:00001c90       ??_C@_0BD@JFADHEFE@Ljava?1lang?1String?$DL@ 0000000180005c90     libredefclass004.obj
 0002:00001ca8       ??_C@_0BC@NKAJJLHG@stringComplNewFld@ 0000000180005ca8     libredefclass004.obj
 0002:00001cc0       ??_C@_0EC@FCFNHCMN@?$CFs?3?5Failed?5to?5get?5the?5field?5ID?5@ 0000000180005cc0     libredefclass004.obj
 0002:00001d08       ??_C@_0BM@LHALNHJF@completely?5new?5String?5field@ 0000000180005d08     libredefclass004.obj
 0002:00001d28       ??_C@_0DP@JPBAGOK@Completely?5new?5fields?5have?5not?5@ 0000000180005d28     libredefclass004.obj
 0002:00001d68       ??_C@_0CD@EEFKBHGF@?7intComplNewFld?5?$DN?5?$CFd?0?7expected?5@ 0000000180005d68     libredefclass004.obj
 0002:00001d90       ??_C@_0BJ@EBJOJCFC@?7longComplNewFld?5?$DN?5?$CFI64d@ 0000000180005d90     libredefclass004.obj
 0002:00001db0       ??_C@_0BC@EEFIOPJN@?0?7expected?5?$CFI64d?6@ 0000000180005db0     libredefclass004.obj
 0002:00001dc8       ??_C@_0CK@FHODDECA@?7stringComplNewFld?5?$DN?5?$CC?$CFs?$CC?0?7expe@ 0000000180005dc8     libredefclass004.obj
 0002:00001e00       ??_C@_0GA@DPEPFGNH@Completely?5new?5fields?3?6?7stringC@ 0000000180005e00     libredefclass004.obj
 0002:00001e70       ??_C@_1EC@JIJBPKFM@?$AAa?$AAp?$AAi?$AA?9?$AAm?$AAs?$AA?9?$AAw?$AAi?$AAn?$AA?9?$AAc?$AAo?$AAr?$AAe@ 0000000180005e70     MSVCRT:thread_safe_statics.obj
 0002:00001eb8       ??_C@_1BK@MGMFAEKH@?$AAk?$AAe?$AAr?$AAn?$AAe?$AAl?$AA3?$AA2?$AA?4?$AAd?$AAl?$AAl@ 0000000180005eb8     MSVCRT:thread_safe_statics.obj
 0002:00001ed8       ??_C@_0BJ@JEBJOJFJ@SleepConditionVariableCS@ 0000000180005ed8     MSVCRT:thread_safe_statics.obj
 0002:00001ef8       ??_C@_0BJ@PGPPEPCC@WakeAllConditionVariable@ 0000000180005ef8     MSVCRT:thread_safe_statics.obj
 0002:00001f18       _pDefaultRawDllMain        0000000180005f18     MSVCRT:dll_dllmain.obj
 0002:00001f18       _pRawDllMain               0000000180005f18     MSVCRT:dll_dllmain.obj
 0002:00001f20       __xmm@ffffffffffffffffffffffffffffffff 0000000180005f20     MSVCRT:utility.obj
 0002:00001f30       _load_config_used          0000000180005f30     MSVCRT:loadcfg.obj
 0002:00002100       _tls_used                  0000000180006100     MSVCRT:tlssup.obj
 0002:00002128       __volatile_metadata        0000000180006128     <linker-defined>
 0002:000024e8       __rtc_iaa                  00000001800064e8     MSVCRT:initsect.obj
 0002:000024f0       __rtc_izz                  00000001800064f0     MSVCRT:initsect.obj
 0002:000024f8       __rtc_taa                  00000001800064f8     MSVCRT:initsect.obj
 0002:00002500       __rtc_tzz                  0000000180006500     MSVCRT:initsect.obj
 0002:00002508       _tls_start                 0000000180006508     MSVCRT:tlssup.obj
 0002:0000250c       _Init_thread_epoch         000000018000650c     MSVCRT:thread_safe_statics.obj
 0002:00002510       _tls_end                   0000000180006510     MSVCRT:tlssup.obj
 0002:00002c14       __IMPORT_DESCRIPTOR_KERNEL32 0000000180006c14     kernel32:KERNEL32.dll
 0002:00002c28       __IMPORT_DESCRIPTOR_VCRUNTIME140 0000000180006c28     vcruntime:VCRUNTIME140.dll
 0002:00002c3c       __IMPORT_DESCRIPTOR_api-ms-win-crt-runtime-l1-1-0 0000000180006c3c     ucrt:api-ms-win-crt-runtime-l1-1-0.dll
 0002:00002c50       __IMPORT_DESCRIPTOR_api-ms-win-crt-stdio-l1-1-0 0000000180006c50     ucrt:api-ms-win-crt-stdio-l1-1-0.dll
 0002:00002c64       __IMPORT_DESCRIPTOR_api-ms-win-crt-string-l1-1-0 0000000180006c64     ucrt:api-ms-win-crt-string-l1-1-0.dll
 0002:00002c78       __NULL_IMPORT_DESCRIPTOR   0000000180006c78     kernel32:KERNEL32.dll
 0003:00000040       _Init_global_epoch         0000000180008040     MSVCRT:thread_safe_statics.obj
 0003:00000050       __security_cookie          0000000180008050     MSVCRT:gs_cookie.obj
 0003:00000058       __security_cookie_complement 0000000180008058     MSVCRT:gs_cookie.obj
 0003:00000060       __scrt_native_dllmain_reason 0000000180008060     MSVCRT:utility.obj
 0003:00000068       __isa_available            0000000180008068     MSVCRT:cpu_disp.obj
 0003:0000006c       __isa_enabled              000000018000806c     MSVCRT:cpu_disp.obj
 0003:00000070       __memset_fast_string_threshold 0000000180008070     MSVCRT:cpu_disp.obj
 0003:00000078       __memset_nt_threshold      0000000180008078     MSVCRT:cpu_disp.obj
 0003:00000080       __scrt_ucrt_dll_is_in_use  0000000180008080     MSVCRT:ucrt_stubs.obj
 0003:00000090       g_wrongHeapCallbacks       0000000180008090     libredefclass004.obj
 0003:00000110       g_szTagInfo                0000000180008110     libredefclass004.obj
 0003:00002050       g_tagFlags                 000000018000a050     libredefclass004.obj
 0003:00002438       g_refsToVerifyCnt          000000018000a438     libredefclass004.obj
 0003:0000243c       g_fakeUserData             000000018000a43c     libredefclass004.obj
 0003:00002440       g_tagVisitCount            000000018000a440     libredefclass004.obj
 0003:000033e0       g_refsToVerify             000000018000b3e0     libredefclass004.obj
 0003:0001aae0       g_userDataError            0000000180022ae0     libredefclass004.obj
 0003:0001ac90       ?_OptionsStorage@?1??__local_stdio_printf_options@@9@4_KA 0000000180022c90     libredefclass004.obj
 0003:0001b258       _tls_index                 0000000180023258     MSVCRT:tlssup.obj
 0003:0001b260       __scrt_current_native_startup_state 0000000180023260     MSVCRT:utility.obj
 0003:0001b268       __scrt_native_startup_lock 0000000180023268     MSVCRT:utility.obj
 0003:0001b2a8       __scrt_debugger_hook_flag  00000001800232a8     MSVCRT:utility_desktop.obj
 0003:0001b2b0       ?__type_info_root_node@@3U__type_info_node@@A 00000001800232b0     MSVCRT:tncleanup.obj
 0003:0001b2c0       ?_OptionsStorage@?1??__local_stdio_scanf_options@@9@4_KA 00000001800232c0     MSVCRT:default_local_stdio_options.obj
 0003:0001b2c8       __favor                    00000001800232c8     MSVCRT:cpu_disp.obj
 0003:0001b2d0       __dyn_tls_init_callback    00000001800232d0     <common>

 entry point at        0001:000024a0

 Static symbols

 0000:fffda000       .debug$S                   0000000180000000     redefclass004.exp
 0000:fffda000       .debug$S                   0000000180000000     vcruntime:VCRUNTIME140.dll
 0000:fffda000       .debug$S                   0000000180000000     vcruntime:VCRUNTIME140.dll
 0000:fffda000       .debug$S                   0000000180000000     vcruntime:VCRUNTIME140.dll
 0000:fffda000       .debug$S                   0000000180000000     vcruntime:VCRUNTIME140.dll
 0000:fffda000       .debug$S                   0000000180000000     vcruntime:VCRUNTIME140.dll
 0000:fffda000       .debug$S                   0000000180000000     vcruntime:VCRUNTIME140.dll
 0000:fffda000       .debug$S                   0000000180000000     vcruntime:VCRUNTIME140.dll
 0000:fffda000       .debug$S                   0000000180000000     ucrt:api-ms-win-crt-convert-l1-1-0.dll
 0002:ffffc000       .idata$6                   0000000180000000     ucrt:api-ms-win-crt-convert-l1-1-0.dll
 0000:fffda000       .debug$S                   0000000180000000     ucrt:api-ms-win-crt-heap-l1-1-0.dll
 0000:fffda000       .debug$S                   0000000180000000     ucrt:api-ms-win-crt-heap-l1-1-0.dll
 0000:fffda000       .debug$S                   0000000180000000     ucrt:api-ms-win-crt-heap-l1-1-0.dll
 0000:fffda000       .debug$S                   0000000180000000     ucrt:api-ms-win-crt-heap-l1-1-0.dll
 0002:ffffc000       .idata$6                   0000000180000000     ucrt:api-ms-win-crt-heap-l1-1-0.dll
 0000:fffda000       .debug$S                   0000000180000000     ucrt:api-ms-win-crt-runtime-l1-1-0.dll
 0000:fffda000       .debug$S                   0000000180000000     ucrt:api-ms-win-crt-runtime-l1-1-0.dll
 0000:fffda000       .debug$S                   0000000180000000     ucrt:api-ms-win-crt-runtime-l1-1-0.dll
 0000:fffda000       .debug$S                   0000000180000000     ucrt:api-ms-win-crt-runtime-l1-1-0.dll
 0000:fffda000       .debug$S                   0000000180000000     ucrt:api-ms-win-crt-runtime-l1-1-0.dll
 0000:fffda000       .debug$S                   0000000180000000     ucrt:api-ms-win-crt-runtime-l1-1-0.dll
 0000:fffda000       .debug$S                   0000000180000000     ucrt:api-ms-win-crt-runtime-l1-1-0.dll
 0000:fffda000       .debug$S                   0000000180000000     ucrt:api-ms-win-crt-runtime-l1-1-0.dll
 0000:fffda000       .debug$S                   0000000180000000     ucrt:api-ms-win-crt-runtime-l1-1-0.dll
 0000:fffda000       .debug$S                   0000000180000000     ucrt:api-ms-win-crt-runtime-l1-1-0.dll
 0000:fffda000       .debug$S                   0000000180000000     ucrt:api-ms-win-crt-runtime-l1-1-0.dll
 0000:fffda000       .debug$S                   0000000180000000     ucrt:api-ms-win-crt-runtime-l1-1-0.dll
 0000:fffda000       .debug$S                   0000000180000000     ucrt:api-ms-win-crt-runtime-l1-1-0.dll
 0000:fffda000       .debug$S                   0000000180000000     ucrt:api-ms-win-crt-runtime-l1-1-0.dll
 0000:fffda000       .debug$S                   0000000180000000     ucrt:api-ms-win-crt-runtime-l1-1-0.dll
 0000:fffda000       .debug$S                   0000000180000000     ucrt:api-ms-win-crt-runtime-l1-1-0.dll
 0000:fffda000       .debug$S                   0000000180000000     ucrt:api-ms-win-crt-stdio-l1-1-0.dll
 0000:fffda000       .debug$S                   0000000180000000     ucrt:api-ms-win-crt-stdio-l1-1-0.dll
 0000:fffda000       .debug$S                   0000000180000000     ucrt:api-ms-win-crt-stdio-l1-1-0.dll
 0000:fffda000       .debug$S                   0000000180000000     ucrt:api-ms-win-crt-stdio-l1-1-0.dll
 0000:fffda000       .debug$S                   0000000180000000     ucrt:api-ms-win-crt-stdio-l1-1-0.dll
 0000:fffda000       .debug$S                   0000000180000000     ucrt:api-ms-win-crt-stdio-l1-1-0.dll
 0000:fffda000       .debug$S                   0000000180000000     ucrt:api-ms-win-crt-stdio-l1-1-0.dll
 0000:fffda000       .debug$S                   0000000180000000     ucrt:api-ms-win-crt-stdio-l1-1-0.dll
 0000:fffda000       .debug$S                   0000000180000000     ucrt:api-ms-win-crt-stdio-l1-1-0.dll
 0000:fffda000       .debug$S                   0000000180000000     ucrt:api-ms-win-crt-stdio-l1-1-0.dll
 0000:fffda000       .debug$S                   0000000180000000     ucrt:api-ms-win-crt-string-l1-1-0.dll
 0000:fffda000       .debug$S                   0000000180000000     ucrt:api-ms-win-crt-string-l1-1-0.dll
 0000:fffda000       .debug$S                   0000000180000000     ucrt:api-ms-win-crt-string-l1-1-0.dll
 0000:fffda000       .debug$S                   0000000180000000     ucrt:api-ms-win-crt-string-l1-1-0.dll
 0000:fffda000       .debug$S                   0000000180000000     ucrt:api-ms-win-crt-string-l1-1-0.dll
 0000:fffda000       .debug$S                   0000000180000000     ucrt:api-ms-win-crt-string-l1-1-0.dll
 0000:fffda000       .debug$S                   0000000180000000     ucrt:api-ms-win-crt-string-l1-1-0.dll
 0000:fffda000       .debug$S                   0000000180000000     ucrt:api-ms-win-crt-string-l1-1-0.dll
 0000:fffda000       .debug$S                   0000000180000000     kernel32:KERNEL32.dll
 0000:fffda000       .debug$S                   0000000180000000     kernel32:KERNEL32.dll
 0000:fffda000       .debug$S                   0000000180000000     kernel32:KERNEL32.dll
 0000:fffda000       .debug$S                   0000000180000000     kernel32:KERNEL32.dll
 0000:fffda000       .debug$S                   0000000180000000     kernel32:KERNEL32.dll
 0000:fffda000       .debug$S                   0000000180000000     kernel32:KERNEL32.dll
 0000:fffda000       .debug$S                   0000000180000000     kernel32:KERNEL32.dll
 0000:fffda000       .debug$S                   0000000180000000     kernel32:KERNEL32.dll
 0000:fffda000       .debug$S                   0000000180000000     kernel32:KERNEL32.dll
 0000:fffda000       .debug$S                   0000000180000000     kernel32:KERNEL32.dll
 0000:fffda000       .debug$S                   0000000180000000     kernel32:KERNEL32.dll
 0000:fffda000       .debug$S                   0000000180000000     kernel32:KERNEL32.dll
 0000:fffda000       .debug$S                   0000000180000000     kernel32:KERNEL32.dll
 0000:fffda000       .debug$S                   0000000180000000     kernel32:KERNEL32.dll
 0000:fffda000       .debug$S                   0000000180000000     kernel32:KERNEL32.dll
 0000:fffda000       .debug$S                   0000000180000000     kernel32:KERNEL32.dll
 0000:fffda000       .debug$S                   0000000180000000     kernel32:KERNEL32.dll
 0000:fffda000       .debug$S                   0000000180000000     kernel32:KERNEL32.dll
 0000:fffda000       .debug$S                   0000000180000000     kernel32:KERNEL32.dll
 0000:fffda000       .debug$S                   0000000180000000     kernel32:KERNEL32.dll
 0000:fffda000       .debug$S                   0000000180000000     kernel32:KERNEL32.dll
 0000:fffda000       .debug$S                   0000000180000000     kernel32:KERNEL32.dll
 0000:fffda000       .debug$S                   0000000180000000     kernel32:KERNEL32.dll
 0000:fffda000       .debug$S                   0000000180000000     kernel32:KERNEL32.dll
 0000:fffda000       .debug$S                   0000000180000000     kernel32:KERNEL32.dll
 0000:fffda000       .debug$S                   0000000180000000     kernel32:KERNEL32.dll
 0000:fffda000       .debug$S                   0000000180000000     kernel32:KERNEL32.dll
 0000:fffda000       .debug$S                   0000000180000000     kernel32:KERNEL32.dll
 0001:000010b4       addRefToVerify             00000001800020b4 f   libredefclass004.obj
 0001:00001120       agentThreadWrapper         0000000180002120 f   libredefclass004.obj
 0001:00001310       file_basename              0000000180002310 f   libredefclass004.obj
 0001:0000197c       startAgentThreadWrapper    000000018000297c f   libredefclass004.obj
 0001:00001cbc       syncDebuggeeStatus         0000000180002cbc f   libredefclass004.obj
 0001:00001f5c       capture_previous_context   0000000180002f5c f   MSVCRT:gs_report.obj
 0001:00001fd0       ?__scrt_initialize_thread_safe_statics@@YAHXZ 0000000180002fd0 f   MSVCRT:thread_safe_statics.obj
 0001:000020a0       ?__scrt_uninitialize_thread_safe_statics@@YAXXZ 00000001800030a0 f   MSVCRT:thread_safe_statics.obj
 0001:00002150       $$000000                   0000000180003150     MSVCRT:amdsecgs.obj
 0001:00002180       ?dllmain_crt_dispatch@@YAHQEAUHINSTANCE__@@KQEAX@Z 0000000180003180 f   MSVCRT:dll_dllmain.obj
 0001:000021d0       ?dllmain_crt_process_attach@@YAHQEAUHINSTANCE__@@QEAX@Z 00000001800031d0 f   MSVCRT:dll_dllmain.obj
 0001:000022e8       ?dllmain_crt_process_detach@@YAH_N@Z 00000001800032e8 f   MSVCRT:dll_dllmain.obj
 0001:0000236c       ?dllmain_dispatch@@YAHQEAUHINSTANCE__@@KQEAX@Z 000000018000336c f   MSVCRT:dll_dllmain.obj
 0001:00002d80       $$000000                   0000000180003d80     MSVCRT:guard_dispatch.obj
 0001:00002da0       $$000000                   0000000180003da0     MSVCRT:guard_xfg_dispatch.obj
 0001:00002db6       ?fin$0@?0??dllmain_crt_process_attach@@YAHQEAUHINSTANCE__@@QEAX@Z@4HA 0000000180003db6 f   MSVCRT:dll_dllmain.obj
 0001:00002dcd       ?fin$0@?0??dllmain_crt_process_detach@@YAH_N@Z@4HA 0000000180003dcd f   MSVCRT:dll_dllmain.obj
 0001:00002de6       ?fin$1@?0??dllmain_crt_process_detach@@YAH_N@Z@4HA 0000000180003de6 f   MSVCRT:dll_dllmain.obj
 0001:00002dfa       ?filt$0@?0??dllmain_dispatch@@YAHQEAUHINSTANCE__@@KQEAX@Z@4HA 0000000180003dfa f   MSVCRT:dll_dllmain.obj
 0001:00002e30       __scrt_is_nonwritable_in_current_image$filt$0 0000000180003e30 f   MSVCRT:utility.obj
 0002:000001e8       ?__scrt_initialize_tss_var@@3P6AHXZEA 00000001800041e8     MSVCRT:thread_safe_statics.obj
 0002:00000310       ?opcLengths@@3QBEB         0000000180004310     libredefclass004.obj
 0002:00001e60       GS_ExceptionPointers       0000000180005e60     MSVCRT:gs_report.obj
 0002:00002518       $unwind$fprintf            0000000180006518     libredefclass004.obj
 0002:00002524       $unwind$printf             0000000180006524     libredefclass004.obj
 0002:00002530       $unwind$?NewObject@JNIEnv_@@QEAAPEAV_jobject@@PEAV_jclass@@PEAU_jmethodID@@ZZ 0000000180006530     libredefclass004.obj
 0002:00002530       $unwind$nsk_lcomplain      0000000180006530     libredefclass004.obj
 0002:00002530       $unwind$nsk_ldisplay       0000000180006530     libredefclass004.obj
 0002:00002538       $unwind$nsk_lvdisplay      0000000180006538     libredefclass004.obj
 0002:00002538       $unwind$_RTC_Initialize    0000000180006538     MSVCRT:initsect.obj
 0002:00002538       $unwind$_RTC_Terminate     0000000180006538     MSVCRT:initsect.obj
 0002:00002538       $unwind$?__scrt_initialize_thread_safe_statics@@YAHXZ 0000000180006538     MSVCRT:thread_safe_statics.obj
 0002:00002544       $unwind$nsk_lvcomplain     0000000180006544     libredefclass004.obj
 0002:0000255c       $unwind$nsk_ltrace         000000018000655c     libredefclass004.obj
 0002:0000255c       $unwind$__report_gsfailure 000000018000655c     MSVCRT:gs_report.obj
 0002:00002564       $unwind$Agent_Initialize   0000000180006564     libredefclass004.obj
 0002:00002564       $unwind$nsk_lvtrace        0000000180006564     libredefclass004.obj
 0002:00002564       $unwind$__raise_securityfailure 0000000180006564     MSVCRT:gs_report.obj
 0002:00002564       $unwind$__scrt_initialize_crt 0000000180006564     MSVCRT:utility.obj
 0002:00002564       $unwind$__scrt_initialize_onexit_tables 0000000180006564     MSVCRT:utility.obj
 0002:00002564       $unwind$__scrt_release_startup_lock 0000000180006564     MSVCRT:utility.obj
 0002:00002564       $unwind$__scrt_uninitialize_crt 0000000180006564     MSVCRT:utility.obj
 0002:00002564       $unwind$_onexit            0000000180006564     MSVCRT:utility.obj
 0002:0000256c       $unwind$nsk_lverify        000000018000656c     libredefclass004.obj
 0002:0000257c       $unwind$nsk_vprintf        000000018000657c     libredefclass004.obj
 0002:0000258c       $unwind$nsk_printf         000000018000658c     libredefclass004.obj
 0002:00002594       $unwind$?nsk_jni_lverify@@YAHHPEAUJNIEnv_@@HQEBDH1ZZ 0000000180006594     libredefclass004.obj
 0002:000025a8       $unwind$?nsk_jni_check_exception@@YAHPEAUJNIEnv_@@QEBDH@Z 00000001800065a8     libredefclass004.obj
 0002:000025c4       $unwind$Java_nsk_jvmti_unit_FollowReferences_FollowRefObjects_resetTags 00000001800065c4     libredefclass004.obj
 0002:000025c4       $unwind$addRefToVerify     00000001800065c4     libredefclass004.obj
 0002:000025c4       $unwind$nsk_jvmti_resetAgentData 00000001800065c4     libredefclass004.obj
 0002:000025c4       $unwind$nsk_jvmti_setFailStatus 00000001800065c4     libredefclass004.obj
 0002:000025c4       $unwind$__scrt_initialize_default_local_stdio_options 00000001800065c4     MSVCRT:default_local_stdio_options.obj
 0002:000025c4       $unwind$?dllmain_crt_dispatch@@YAHQEAUHINSTANCE__@@KQEAX@Z 00000001800065c4     MSVCRT:dll_dllmain.obj
 0002:000025c4       $unwind$DllMain            00000001800065c4     MSVCRT:dll_dllmain_stub.obj
 0002:000025c4       $unwind$__GSHandlerCheck   00000001800065c4     MSVCRT:gshandler.obj
 0002:000025c4       $unwind$?__scrt_uninitialize_thread_safe_statics@@YAXXZ 00000001800065c4     MSVCRT:thread_safe_statics.obj
 0002:000025c4       $unwind$__scrt_acquire_startup_lock 00000001800065c4     MSVCRT:utility.obj
 0002:000025c4       $unwind$__scrt_dllmain_after_initialize_c 00000001800065c4     MSVCRT:utility.obj
 0002:000025c4       $unwind$__scrt_dllmain_before_initialize_c 00000001800065c4     MSVCRT:utility.obj
 0002:000025c4       $unwind$__scrt_dllmain_crt_thread_attach 00000001800065c4     MSVCRT:utility.obj
 0002:000025c4       $unwind$__scrt_dllmain_crt_thread_detach 00000001800065c4     MSVCRT:utility.obj
 0002:000025c4       $unwind$__scrt_dllmain_uninitialize_c 00000001800065c4     MSVCRT:utility.obj
 0002:000025c4       $unwind$__scrt_dllmain_uninitialize_critical 00000001800065c4     MSVCRT:utility.obj
 0002:000025c4       $unwind$atexit             00000001800065c4     MSVCRT:utility.obj
 0002:000025cc       $unwind$nsk_jvmti_lverify  00000001800065cc     libredefclass004.obj
 0002:000025e0       $unwind$exitOnError        00000001800065e0     libredefclass004.obj
 0002:000025f0       $unwind$Java_nsk_share_jvmti_ArgumentHandler_getAgentOptionsString 00000001800065f0     libredefclass004.obj
 0002:00002604       $unwind$Java_nsk_jvmti_unit_FollowReferences_FollowRefObjects_getTag 0000000180006604     libredefclass004.obj
 0002:00002604       $unwind$Java_nsk_share_jvmti_DebugeeClass_checkStatus 0000000180006604     libredefclass004.obj
 0002:00002604       $unwind$agentThreadWrapper 0000000180006604     libredefclass004.obj
 0002:00002614       $unwind$startAgentThreadWrapper 0000000180006614     libredefclass004.obj
 0002:00002630       $unwind$syncDebuggeeStatus 0000000180006630     libredefclass004.obj
 0002:00002630       $unwind$__scrt_dllmain_exception_filter 0000000180006630     MSVCRT:utility.obj
 0002:00002644       $unwind$Java_nsk_share_jvmti_DebugeeClass_resetAgentData 0000000180006644     libredefclass004.obj
 0002:0000264c       $unwind$MA_checkStatus     000000018000664c     libredefclass004.obj
 0002:00002660       $unwind$Java_nsk_jvmti_unit_FollowReferences_FollowRefObjects_setTag 0000000180006660     libredefclass004.obj
 0002:00002678       $unwind$Java_nsk_jvmti_unit_FollowReferences_FollowRefObjects_addRefToVerify 0000000180006678     libredefclass004.obj
 0002:00002694       $unwind$Java_nsk_jvmti_RedefineClasses_redefclass004_makeRedefinition 0000000180006694     libredefclass004.obj
 0002:000026a4       $unwind$Java_nsk_jvmti_RedefineClasses_redefclass004_checkNewFields 00000001800066a4     libredefclass004.obj
 0002:000026c0       $unwind$capture_previous_context 00000001800066c0     MSVCRT:gs_report.obj
 0002:000026cc       $unwind$__GSHandlerCheckCommon 00000001800066cc     MSVCRT:gshandler.obj
 0002:000026d8       $xdatasym                  00000001800066d8     MSVCRT:amdsecgs.obj
 0002:000026dc       $unwind$?dllmain_crt_process_attach@@YAHQEAUHINSTANCE__@@QEAX@Z 00000001800066dc     MSVCRT:dll_dllmain.obj
 0002:00002718       $unwind$?fin$0@?0??dllmain_crt_process_attach@@YAHQEAUHINSTANCE__@@QEAX@Z@4HA 0000000180006718     MSVCRT:dll_dllmain.obj
 0002:00002718       $unwind$?fin$0@?0??dllmain_crt_process_detach@@YAH_N@Z@4HA 0000000180006718     MSVCRT:dll_dllmain.obj
 0002:00002718       $unwind$?fin$1@?0??dllmain_crt_process_detach@@YAH_N@Z@4HA 0000000180006718     MSVCRT:dll_dllmain.obj
 0002:00002720       $unwind$?dllmain_crt_process_detach@@YAH_N@Z 0000000180006720     MSVCRT:dll_dllmain.obj
 0002:00002774       $unwind$?dllmain_dispatch@@YAHQEAUHINSTANCE__@@KQEAX@Z 0000000180006774     MSVCRT:dll_dllmain.obj
 0002:0000279c       $unwind$?filt$0@?0??dllmain_dispatch@@YAHQEAUHINSTANCE__@@KQEAX@Z@4HA 000000018000679c     MSVCRT:dll_dllmain.obj
 0002:000027a4       $unwind$_DllMainCRTStartup 00000001800067a4     MSVCRT:dll_dllmain.obj
 0002:000027b4       $unwind$__scrt_is_nonwritable_in_current_image 00000001800067b4     MSVCRT:utility.obj
 0002:000027d4       $unwind$__scrt_is_nonwritable_in_current_image$filt$0 00000001800067d4     MSVCRT:utility.obj
 0002:000027dc       $unwind$__scrt_fastfail    00000001800067dc     MSVCRT:utility_desktop.obj
 0002:000027ec       $unwind$__security_init_cookie 00000001800067ec     MSVCRT:gs_support.obj
 0002:000027f8       $unwind$__isa_available_init 00000001800067f8     MSVCRT:cpu_disp.obj
 0002:00002808       $xdatasym                  0000000180006808     MSVCRT:guard_dispatch.obj
 0002:00002810       $xdatasym                  0000000180006810     MSVCRT:guard_xfg_dispatch.obj
 0002:00002820       .edata                     0000000180006820     redefclass004.exp
 0002:00002848       rgpv                       0000000180006848     redefclass004.exp
 0002:00002888       rgszName                   0000000180006888     redefclass004.exp
 0002:000028c8       rgwOrd                     00000001800068c8     redefclass004.exp
 0002:000028e8       szName                     00000001800068e8     redefclass004.exp
 0002:000028fa       $N00001                    00000001800068fa     redefclass004.exp
 0002:00002909       $N00002                    0000000180006909     redefclass004.exp
 0002:00002916       $N00003                    0000000180006916     redefclass004.exp
 0002:00002952       $N00004                    0000000180006952     redefclass004.exp
 0002:00002990       $N00005                    0000000180006990     redefclass004.exp
 0002:000029d5       $N00006                    00000001800069d5     redefclass004.exp
 0002:00002a12       $N00007                    0000000180006a12     redefclass004.exp
 0002:00002a5a       $N00008                    0000000180006a5a     redefclass004.exp
 0002:00002a9a       $N00009                    0000000180006a9a     redefclass004.exp
 0002:00002ad7       $N00010                    0000000180006ad7     redefclass004.exp
 0002:00002b12       $N00011                    0000000180006b12     redefclass004.exp
 0002:00002b40       $N00012                    0000000180006b40     redefclass004.exp
 0002:00002b71       $N00013                    0000000180006b71     redefclass004.exp
 0002:00002ba0       $N00014                    0000000180006ba0     redefclass004.exp
 0002:00002bcf       $N00015                    0000000180006bcf     redefclass004.exp
 0002:00002c04       $N00016                    0000000180006c04     redefclass004.exp
 0002:00003012       .idata$6                   0000000180007012     kernel32:KERNEL32.dll
 0002:00003076       .idata$6                   0000000180007076     vcruntime:VCRUNTIME140.dll
 0002:000031e2       .idata$6                   00000001800071e2     ucrt:api-ms-win-crt-runtime-l1-1-0.dll
 0002:00003204       .idata$6                   0000000180007204     ucrt:api-ms-win-crt-stdio-l1-1-0.dll
 0002:00003224       .idata$6                   0000000180007224     ucrt:api-ms-win-crt-string-l1-1-0.dll
 0003:00000000       ?codeAttributeName@@3PEBDEB 0000000180008000     libredefclass004.obj
 0003:00000008       ?lineNumberAttributeName@@3PEBDEB 0000000180008008     libredefclass004.obj
 0003:00000010       ?localVarAttributeName@@3PEBDEB 0000000180008010     libredefclass004.obj
 0003:00000018       ?localVarTypeAttributeName@@3PEBDEB 0000000180008018     libredefclass004.obj
 0003:00000020       ?stackMapAttributeName@@3PEBDEB 0000000180008020     libredefclass004.obj
 0003:00000028       ?callBytes@@3PAEA          0000000180008028     libredefclass004.obj
 0003:0000002c       ?allocBytes@@3PAEA         000000018000802c     libredefclass004.obj
 0003:00000030       INTFLD                     0000000180008030     libredefclass004.obj
 0003:00000038       LONGFLD                    0000000180008038     libredefclass004.obj
 0003:0001aae4       redefineAttempted          0000000180022ae4     libredefclass004.obj
 0003:0001aae8       nsk_context                0000000180022ae8     libredefclass004.obj
 0003:0001aaf4       redefineSucceed            0000000180022af4     libredefclass004.obj
 0003:0001aaf8       agentFailed                0000000180022af8     libredefclass004.obj
 0003:0001aafc       currentAgentStatus         0000000180022afc     libredefclass004.obj
 0003:0001ab00       context                    0000000180022b00     libredefclass004.obj
 0003:0001abb8       agentThread                0000000180022bb8     libredefclass004.obj
 0003:0001abc0       agentThreadProc            0000000180022bc0     libredefclass004.obj
 0003:0001abc8       agentThreadArg             0000000180022bc8     libredefclass004.obj
 0003:0001abd0       agent_data                 0000000180022bd0     libredefclass004.obj
 0003:0001abe0       jvmti_env                  0000000180022be0     libredefclass004.obj
 0003:0001abe8       jvm                        0000000180022be8     libredefclass004.obj
 0003:0001abf0       jni_env                    0000000180022bf0     libredefclass004.obj
 0003:0001abf8       checkStatus_func           0000000180022bf8     libredefclass004.obj
 0003:0001ac00       ?codeAttributeIndex@@3GA   0000000180022c00     libredefclass004.obj
 0003:0001ac04       ?lineNumberAttributeIndex@@3GA 0000000180022c04     libredefclass004.obj
 0003:0001ac08       ?localVarAttributeIndex@@3GA 0000000180022c08     libredefclass004.obj
 0003:0001ac0c       ?localVarTypeAttributeIndex@@3GA 0000000180022c0c     libredefclass004.obj
 0003:0001ac10       ?stackMapAttributeIndex@@3GA 0000000180022c10     libredefclass004.obj
 0003:0001ac14       ?stackFrameOffset@@3GA     0000000180022c14     libredefclass004.obj
 0003:0001ac18       ?mode@@3HA                 0000000180022c18     libredefclass004.obj
 0003:0001ac1c       ?constantPoolSize@@3GA     0000000180022c1c     libredefclass004.obj
 0003:0001ac20       ?orig@@3PEBEEB             0000000180022c20     libredefclass004.obj
 0003:0001ac28       ?gen@@3PEAEEA              0000000180022c28     libredefclass004.obj
 0003:0001ac30       ?inputPos@@3PEAEEA         0000000180022c30     libredefclass004.obj
 0003:0001ac38       ?endPos@@3PEBEEB           0000000180022c38     libredefclass004.obj
 0003:0001ac40       ?genPos@@3PEAEEA           0000000180022c40     libredefclass004.obj
 0003:0001ac48       ?markPos@@3PEAEEA          0000000180022c48     libredefclass004.obj
 0003:0001ac50       ?constantPool@@3PEAPEADEA  0000000180022c50     libredefclass004.obj
 0003:0001ac58       ?constantPoolCount@@3GA    0000000180022c58     libredefclass004.obj
 0003:0001ac5c       ?zeroBytes@@3PAEA          0000000180022c5c     libredefclass004.obj
 0003:0001ac60       ?codeLength@@3IA           0000000180022c60     libredefclass004.obj
 0003:0001ac68       ?map@@3PEAIEA              0000000180022c68     libredefclass004.obj
 0003:0001ac70       ?widening@@3PEACEA         0000000180022c70     libredefclass004.obj
 0003:0001ac78       jvmti                      0000000180022c78     libredefclass004.obj
 0003:0001ac80       caps                       0000000180022c80     libredefclass004.obj
 0003:0001aca0       GS_ExceptionRecord         0000000180022ca0     MSVCRT:gs_report.obj
 0003:0001ad40       GS_ContextRecord           0000000180022d40     MSVCRT:gs_report.obj
 0003:0001b210       ?g_tss_cv@@3U_RTL_CONDITION_VARIABLE@@A 0000000180023210     MSVCRT:thread_safe_statics.obj
 0003:0001b218       ?g_tss_event@@3PEAXEA      0000000180023218     MSVCRT:thread_safe_statics.obj
 0003:0001b220       ?g_tss_mutex@@3U_RTL_CRITICAL_SECTION@@A 0000000180023220     MSVCRT:thread_safe_statics.obj
 0003:0001b248       ?g_sleep_condition_variable_cs@@3P6AHPEAU_RTL_CONDITION_VARIABLE@@PEAU_RTL_CRITICAL_SECTION@@K@ZEA 0000000180023248     MSVCRT:thread_safe_statics.obj
 0003:0001b250       ?g_wake_all_condition_variable@@3P6AXPEAU_RTL_CONDITION_VARIABLE@@@ZEA 0000000180023250     MSVCRT:thread_safe_statics.obj
 0003:0001b25c       ?__proc_attached@@3HA      000000018002325c     MSVCRT:dll_dllmain.obj
 0003:0001b270       ?is_initialized_as_dll@@3_NA 0000000180023270     MSVCRT:utility.obj
 0003:0001b271       ?module_local_atexit_table_initialized@@3_NA 0000000180023271     MSVCRT:utility.obj
 0003:0001b278       ?module_local_atexit_table@@3U_onexit_table_t@@A 0000000180023278     MSVCRT:utility.obj
 0003:0001b290       ?module_local_at_quick_exit_table@@3U_onexit_table_t@@A 0000000180023290     MSVCRT:utility.obj
